:0600000000F08CEF1FF080
:023ED200FFFFF0
:103ED500313200FFFF95681200FFFFFFFFFFFFACC7
:103EE50084810EAF6EAC98AB8E948C948EAC8A1296
:103EF50000FFFFFFFF016EFFFFACA284EF1FF087FD
:103F0500EF1FF0FFFF7EEF1FF0FFFF01C0ADFF12B7
:103F150000FFFFD50EF66E3E0EF76E000EF86E0929
:103F250000F5CF0DF00900F5CF0EF00900F5CF0F24
:103F3500F00001C4EF1FF0FFFF000E056E000E0438
:103F45006EB1EF1FF0FFFF04500224D96E05500338
:103F550020DA6EDF507CEC1FF0044A052AFFFF04CF
:103F6500500224D96E05500320DA6EDF50D8A4BE66
:103F7500EF1FF0C1EF1FF0FFFFA5EF1FF0FFFF12CE
:103F850000FFFFFFFF6CEC1FF0000E0C6E000E0B28
:103F95006E71EC1FF00DC008F00EC009F00FC00ADD
:103FA500F0FFFF0E0E076E540E066E460EFFFFE87D
:103FB5002EFDD7062EFBD7072EF9D7080E026E0069
:103FC5000E036E9EEC1FF00B4A0C2A0A0E0B180C02
:103FD50010D8A4F0EF1FF0F3EF1FF0FFFFD3EF1F92
:103FE500F0FFFF360E086E350E096E000E0C6E00E2
:0B3FF5000E0B6ED3EF1FF001EF00F089
:020000040020DA
:08000000FFFFFFFFFFFFFFFF00
:020000040030CA
:0E000000FF220D0EFF0080FF0FC00FE00F402B
:00000001FF
